S12301007E02062853294554204F522028472945542054494D453F040A0D5345434F4E44A1
S123012053205B30302D35395D0A0D040A0D4D494E55544553205B30302D35395D0A0D0450
S12301400A0D484F555253205B30302D32335D0A0D040A0D444159204F46205745454B20F8
S12301605B30312D30372C204D4F4E3D30312053554E3D30375D0A0D040A0D4441544520D0
S12301805B30312D33315D0A0D040A0D4D4F4E5448205B30312D31325D0A0D040A0D594560
S12301A04152205B303030302D393939395D0A0D040A0D434F52524543543F205B43523D2F
S12301C05945535D0A0D040A0D41424F525445440A0D040A0D54494D45205345540A0D0412
S11F01E04D4F4E04545545045745440454485504465249045341540453554E047B
S1230206CE0103BDC009BD7FEB84DF8147270D815327037EC000BD02D0BDC021BD02A8B670
S123022601FCB1020527F5B70205860DBDC003BDC024B601FF4AC6043DCE01E03ABDC009FB
S1230246BDC024CE0204BDC0120909098608BDC003BDC01209098608BDC003862DBDC00385
S1230266BDC01209098608BDC003862DBDC003BDC012090909BDC01209098608BDC00386B3
S12302863ABDC003BDC01209098608BDC003863ABDC003BDC012BD7FE54D2780BD7FEB7E62
S12302A6C00086009702BD036EC668BD03C34FB701FCCE01FC5FBD0409C668BD0393C60830
S12302C6CE01FCBD03E9BD03DE39CE019CBDC009BDC01E18B70204F70202CE018ABDC0098E
S12302E6BDC01B841FB70201CE0179BDC009BDC01B843FB70200CE0152BDC009BDC01B845A
S123030607B701FFCE0140BDC009BDC01B843FB701FECE012CBDC009BDC01B847FB701FD9E
S1230326CE0118BDC009BDC01B847FB701FC7F0203CE01B1BDC009BD7FEB810D2708CE01BA
S1230346C7BDC009202186009702BD036EC668BD03C37F0205CE02055FBD0409CE01FCC6F2
S123036608BD0409BD03DE398680B780518655B7805086A0B780518600B7805086C1B780A1
S123038651BD038B39B68051840127F939B680512A10BD038B58CA01F7805086C5B7805150
S12303A6200B8645B7805158CA01F78050B680512BFB84082605B680500D390C39BD038B0B
S12303C658C4FEF7805086C5B78051B680512BFB840826020D390C39B680512BFB86C3B7C6
S12303E6805139B680512BFB840826155D26058640B78051B68050A700085AC1FF26E40D39
S11E0406390C39A60008B78050B680512BFB840826075AC1FF26EC0D390C3907
S9030000FC
